S31508001800000A0020D9180008E7180008E918000897
S3150800181000000000000000000000000000000000BA
S315080018200000000000000000000000000119000888
S31508001830000000000000000003190008D93700085E
S31508001840E5420008071900080719000807190008E3
S3150800185007190008071900080719000807190008DA
S31508001860071900089528000807190008071900082D
S3150800187007190008071900080719000807190008BA
S3150800188007190008000000000000000007190008FA
S3150800189000000000071900080719000807190008C2
S315080018A0000000000719000807190008053D000890
S315080018B007190008071900080719000800000000A2
S315080018C0EE11AA550348854600F0B2FC00480047C9
S315080018D0AD500008000A00200B4880F308880B4822
S315080018E080470B480047FEE704207146084202D0AD
S315080018F0EFF3098001E0EFF30880714603F0CCFAB4
S31508001900FEE7FEE7FEE7FEE7000A00205539000875
S31508001910C518000830B50B460146002020220124D0
S3150800192009E00D46D5409D4205D31D469540491B05
S315080019302546954040191546521E002DF1DC30BD4E
S3150800194070B500242546002801DA01244042002902
S3150800195001DA01254942FFF7DDFFAC4200D04042DB
S31508001960002C00D0494270BD03460B439B0703D0A9
S3150800197009E008C9121F08C0042AFAD203E00B7846
S315080019800370401C491C521EF9D27047D2B201E0BE
S315080019900270401C491EFBD270470022F6E710B5BC
S315080019A013460A4604461946FFF7F0FF204610BDBF
S315080019B0F8B502464A40D40F42004B0052085B086D
S315080019C09A4202D20246084611464A0023D0C30D5F
S315080019D04A00DDB2120EAD1A202D35DA490201266B
S315080019E0490AF6058A19002C00D0524220214F1BBD
S315080019F01146B9402A411018C20D9A4221D0002C2E
S31508001A0017D0012D08DCDA05801AD20F8019D20703
S31508001A10DBB200F023FBF8BDDA05801A012340008B
S31508001A201B06C01880185A428018CA0F104349006E
S31508001A3007E04908C2071143DA05801A80194008E9
S31508001A40801800F003FBF8BD61000122511A001B43
S31508001A50F7E70122D2075140AAE70122D2075040F0
S31508001A60A6E7024670B54A40D30FDB0740002DD0E3
S31508001A704A002AD0010E140E000212020919400A61
S31508001A80520A8418E50104465443000A120A2E0431
S31508001A905043A4194219200CC543AA18120C012553
S31508001AA0AD03521C521912047F39240400D0521C6B
S31508001AB0104301D44000491EC2B20C06C0092018C2
S31508001AC0401C4008802A02D003E0002070BD400870
S31508001AD04000002900DA0020184370BD70B50246A0
S31508001AE04A40D50F40004A00ED0740085208002832
S31508001AF014D0002A12D0C40DD30D41020120C0050E
S31508001B005202490A520AE41A091812187D349142F7
S31508001B1001D3641C00E04900002C01DA002070BDE6
S31508001B200023914201D3891A03434008490000283B
S31508001B30F7D100290AD0914202D10121C90705E04F
S31508001B40914201D2012101E00121C943E005C018F3
S31508001B50401900F07BFA70BDF0B5074608465840B4
S31508001B6087B0C00F049048000E465900400849083F
S31508001B70BC1A884105D2384631461E4617460B46DA
S31508001B8002465800400810434CD0300D03904005DB
S31508001B905900400D490D0590401A0290402872DA06
S31508001BA018030121000B09050843019004980092C7
S31508001BB0002805D0019952420020884100920190E0
S31508001BC0029840210A1A0199009800F00BFA054676
S31508001BD00C466B4607CB00F026FAC0197141039AEA
S31508001BE00E0D0023D71756401A467A40164344D09E
S31508001BF0049A002A2DD0029A012A039A15DC1205A6
S31508001C00C01A914101263605001C7141D20F059E66
S31508001C10D2070093019202962A46234600F064FAF8
S31508001C2007B0F0BD38463146FAE71605224A0F4690
S31508001C30B218C01AB74101210905001C4F41001806
S31508001C407F41114618187941E20F10436D19644116
S31508001C5013E0E2076D0815436408C2071443039AA4
S31508001C6001261205C01A91413605001C7141CE079E
S31508001C70400830434908C01851412A46234600F017
S31508001C8026FACDE7FFE7049801224000C117121A89
S31508001C9000238B4104983146C417381AA141EEE750
S31508001CA030B40124E407634030BC55E730B401245E
S31508001CB0E407614030BC4FE70000E0FFF0B51FB411
S31508001CC088B00B990998002448400999C00F490023
S31508001CD049080991C0070B990090490049080B91DA
S31508001CE009990898A64608431CD00B990A980843F0
S31508001CF018D0099801244000420D4800410D099862
S31508001D0024050003000B204309900B980003000BE1
S31508001D1020430B9050181C49401800220190144685
S31508001D20104605E0002001460DB0F0BD032801DA93
S31508001D30034600E003239C46C11A0AAE0AE05F0088
S31508001D4008ADED5B4F00F75B7D430027AA187C4181
S31508001D50491C5B1E6145F2DD410004AB5A52210461
S31508001D60120C0A43240C401C0828DFDB0198029059
S31508001D700099704601910090059B049A0799069868
S31508001D8000F0B2F9D0E700000DFCFFFFF0B50C46F5
S31508001D905C4085B0E40FE40703944C000026640811
S31508001DA059009446490802460296224321D06246C3
S31508001DB00A431ED06200570D4A000E032303550D31
S31508001DC0012402462C492405781B1B0B360B4018A8
S31508001DD023432643614600901C46501AB44103D358
S31508001DE00098401C009002E0921800985B41002879
S31508001DF003DA0020014605B0F0BD002001210905DF
S31508001E000746864611E064461D46141BB54106D3AF
S31508001E106546521BB341744607430C43A646CD0795
S31508001E2040084908284392185B4105460D43EAD104
S31508001E301046184313D0604619465040714008436F
S31508001E4006D06046101AB34106D20122002306E0E6
S31508001E5000220123DB0702E00122D2435310009837
S31508001E6074460105381C6141029C039D00196941AD
S31508001E7000F02DF9BFE70000FD030000C217C10FEF
S31508001E80504010B54018CA079623002100F0E6F81E
S31508001E9010BD10B500229623114600F0DFF810BDDC
S31508001EA00EB5C217C10F5040CA0740180021054B8E
S31508001EB00293019200910A460B4600F015F903B009
S31508001EC000BD0000330400000EB50549029100214B
S31508001ED000910A460B46019100F006F903B000BDD1
S31508001EE033040000410040020122400AD205090ECF
S31508001EF080187F2901DA00207047962903DC96228C
S31508001F00511AC84070479639884070474A000903F5
S31508001F100123090B1B051943094B10B5520D9A42AB
S31508001F2001DA002010BD064B34339A4203DC9A1AB4
S31508001F3000F068F810BD03495118884010BD00002C
S31508001F40FF030000CDFBFFFFC20FD2074000400889
S31508001F500BD0C10D0723DB01C91840020905400A49
S31508001F601143C208400711437047002001467047D5
S31508001F7010B5002904DB0124E40740428C412146C0
S31508001F80002B04DB1C460123DB075242A3418B428C
S31508001F9000D1824210BD0000CB0FDB07490010B507
S31508001FA0490802460A4307D00A0D07240903E40133
S31508001FB0090B121B002A01DC002010BDC900440FC2
S31508001FC00C43C100E018D205801800F03FF810BD98
S31508001FD00122D207002800DB101A002900DB511A5B
S31508001FE08142704710B5202A04DB0146203A914009
S31508001FF0002010BD914020239C1A0346E340194354
S31508002000904010BD10B5202A04DB0846203AD0407F
S31508002010002110BD0B46D340D0402024A21A91407F
S315080020200843194610BD10B5202A06DBCB1708460B
S31508002030203A1041C1170B4306E00B461341D04026
S315080020402024A21A91400843194610BD002904DA33
S31508002050401C490001D140084000704770B4002474
S31508002060050C05D11024000402D1002921D0112421
S31508002070050E01D100020834050F01D10001241D07
S31508002080850F01D18000A41C002801DB4000641CD8
S31508002090002908D020252E1B0D46F540A14000D06A
S315080020A001212943084301061B1B000ADB1D02D533
S315080020B0002070BC7047DB05181880180029F8DA6C
S315080020C0401C4900F5D170BC40084000704710B567
S315080020D0002B08DA0024401C614192185B411A4320
S315080020E001D14008400010BDF0B51FB482B00546C6
S315080020F00C0003D0084602F051F902E002F04EF94E
S3150800210020300246009021462846FFF76BFF049BC5
S31508002110059A04460F4618431143084314D0184637
S3150800212010431BD0009840210A1A18460599FFF754
S3150800213069FF05460E46009A05990498FFF752FF6F
S31508002140084305D0012004E02046394607B0F0BD13
S315080021500020C11705430E432C43374300990E98B8
S315080021606305401A7905E40A00220C43FD0A0A3081
S3150800217002D500200146E9E70105101969410C9CC2
S315080021800D9D00196941FFF7A2FFDFE7FEB50023A1
S315080021901A461B1A8A4103DB0020014603B0F0BD2C
S315080021A04A000D0301212D0B0905520D0D43D107D8
S315080021B002D100186D41521E5110FF31FF31013115
S315080021C0002704463E4638460097019102460121FB
S315080021D000200905FFF716FFC3197141F8183246A2
S315080021E084468E464A4161462846611A904104D380
S315080021F06046241A954176461F46241900986D4173
S31508002200401C00903428E1DDF91930467041091B5D
S31508002210A84103D20022D243134601E00022134606
S3150800222001980105381C7141FFF751FFB6E7000018
S31508002230064C0125064E05E0E36807CC2B430C3C0B
S3150800224098471034B442F7D3FFF740FBA46600085A
S31508002250C466000810B50446002C08D101210920DF
S31508002260C00600F0E3FD002000F0E6F852E0012C7D
S3150800227005D102210920C00600F0D8FD4AE0022C4B
S3150800228005D104210920C00600F0D0FD42E0032C48
S3150800229005D108210920C00600F0C8FD3AE0042C43
S315080022A005D110210920C00600F0C0FD32E0052C3A
S315080022B005D120210920C00600F0B8FD2AE0062C29
S315080022C005D140210920C00600F0B0FD22E0072C08
S315080022D005D180210920C00600F0A8FD1AE0082CC7
S315080022E004D101210D4800F0A1FD13E0092C04D109
S315080022F002210A4800F09AFD0CE00B2C04D11021AB
S31508002300064800F093FD05E00C2C03D18021034814
S3150800231000F08CFD204600F08FF810BD0004004840
S315080023207FB500200090019002900390002427E0DA
S3150800233000250CE0E800294940186100405AA10030
S315080023406A4651584018A1005050681C85B2142D91
S31508002350F0DBA1006A4650581421FFF7DBFA282162
S31508002360484361001E4A515A3C225143461864218B
S315080023703046FFF7CFFA6100194A5052601C84B202
S31508002380042CD5DB1748407A002826D01448408804
S315080023901549884203DC1248808888420ADD1148BC
S315080023A02038C07A002805D11049486001210D4817
S315080023B02038C1720A4840880A2803DB0848808802
S315080023C00A280ADA07482038C07A002805D10749BA
S315080023D04860012103482038C1727FBD48040020A7
S315080023E03C010020C0030020E60F0000C0010020C9
S315080023F000B587B001A800F0AFF80121480201F046
S315080024005DF8002001907020029001208002039060
S3150800241000200690059001A9064800F031F8012130
S31508002420044800F021F80121024800F011F807B02D
S3150800243000BD00000024014010B504460723002211
S315080024402146024800F038F810BD0000002401407B
S31508002450002904D0426801231A43426003E0426817
S315080024605208520042607047002904D08268082347
S315080024701A43826003E0826808239A4382607047A1
S3150800248042680B4B1A4042600B684A681A43436815
S315080024901A4342608268074B1A4082600B694A6990
S315080024A01A438B681A4383681A4382607047000090
S315080024B00FBCFFFF8FF1F9FFF0B504460D4616462F
S315080024C01F463F073F0F2B46082B0FD91B071B0F2D
S315080024D0083B606F9A000F21914088436067606FE0
S315080024E099003A468A40104360670BE0206F9A00CD
S315080024F00F21914088432067206F99003A468A4009
S3150800250010432067E0680121A9408843E060E0683D
S315080025100121A9400843E0600120800328400028E3
S3150800252003D0012000F020F807E00120C00328406E
S31508002530002802D0012000F017F8F0BD002905D0C8
S315080025408268FF2301331A43826004E08268FF230E
S3150800255001339A43826070470021016041608160BF
S315080025600173016141617047002806D00649496830
S315080025700C221143044A516005E0034949680C22BC
S315080025809143014A516070470024014010B5244820
S315080025900078012834D10020214908702149088093
S315080025A012E02048008840001F49085A1F49098838
S315080025B0C9001F4A89181B4A1288520088521948AE
S315080025C00088401C17490880164800880428E8DB5C
S315080025D07E2001F093FE022000F02EF90121154815
S315080025E0FFF7ACFF11480088401C104908800846D0
S315080025F00088142804DB0020088001200E49087092
S315080026000D480078002806D0FFF78AFE00200A4900
S31508002610087000F055FC7E2001F070FE10BD000029
S315080026204C010020660100201004002068010020EB
S31508002630480400200024014044010020FFB583B06F
S315080026400C46029400200190002726E000261CE094
S31508002650721C039951430846791CFFF75BF9054636
S31508002660A54201D9281B00E0601B05460298A8422E
S3150800267004D90295059806700698077002980028EE
S3150800268002D10120019002E0761C402EE0D300BF63
S315080026900198002800D002E07F1C042FD6D300BF83
S315080026A0029807B0F0BD000000BF00BF00BF00BF22
S315080026B000BFBFF34F8F00BF00BF00BF06480749E2
S315080026C0C86000BF00BF00BFBFF34F8F00BF00BF89
S315080026D000BF00BF00BFFDE70400FA0500ED00E0FB
S315080026E010B500F001F810BD10B523480078002891
S315080026F017D1224800F06AFF01283CD11F4800780C
S31508002700002838DD1D480078402834DC01F0CDFA71
S315080027101B490860012018490870002019490870EB
S3150800272029E0164A17490978491C501800F04EFF47
S31508002730012816D113480078401C124908700F4822
S3150800274000780978884216D100200B4908700B4892
S315080027504078FF280FD10B48007802280BD1FFF7E5
S31508002760A3FF01F0A2FA064909686431884202D932
S3150800277000200149087010BD15010020CC03002077
S31508002780180100201401002010B586B00446012166
S31508002790880300F093FE0121480400F06FFE012231
S315080027A00921C80600F02DFB01220A210920C006CE
S315080027B000F027FB01A801F07EFB01943021684652
S315080027C0018100214181818101821821C18101A9EC
S315080027D0184801F02DFB0121164801F006FB05A853
S315080027E000F065FB01214902684681820121817555
S315080027F01821C17505A90920C00600F0B5FA0121FE
S315080028008902684681824821C17505A90920C00642
S3150800281000F0AAFA1B2168460170032141700121C4
S31508002820817000F0F7FD01220221024801F0F5FA55
S3150800283006B010BD0038014001B50449009808608B
S3150800284000BF024800680028FBD108BD1C01002013
S31508002850014600220E4B1A61CA005A6100229A618B
S3150800286005221A6100BF0A4A1069C207D20F002A58
S3150800287004D0012212040240002AF4D0044A126944
S3150800288052085200024B1A6100229A6170470000F2
S3150800289000E000E010B500210448FFF74FFE0220D3
S315080028A000F04AF801200249087010BD00240140D2
S315080028B04C01002000B589B00121084600F0DEFD74
S315080028C01A4800F045F801A800F08EF8184801905B
S315080028D0184802900021684601730420049068464F
S315080028E00175802141754900C18289000183202133
S315080028F08176090281830021C183018401A90B48DD
S3150800290000F04CF80121094800F01CF801220221C8
S31508002910064800F039F8092168460170022141701D
S315080029200121817000F076FD09B000BD0800024063
S315080029300024014010040020014948607047000047
S31508002940000002400268520852000A4302607047BB
S3150800295010B504462068400840002060002020602A
S315080029606060A060E060E1B2084608380521FEF71D
S31508002970D1FF01460F2088400249496808430149AA
S31508002980486010BD00000240002A03D003680B43CC
S31508002990036002E003688B430360704710B50A7A48
S315080029A08B7D1A430B7C1A434B7C1A434B8A1A437A
S315080029B08B8A1A430B8B1A434B8B1A430368094CB1
S315080029C023401A43026002680123DB039A438B8B78
S315080029D01A430260CA6842600A6882604A68C2602E
S315080029E010BD00000F80FFFF0021016041600172E9
S315080029F0C16001744174418281828175018341837A
S31508002A008183704770B506460C4621460A4800F091
S31508002A104BF90546002D01D1401E70BD064885427A
S31508002A2002D10648051B00E02D1B224629463046E2
S31508002A30FEF79AFF2046F0E700F4000800FC0008BD
S31508002A4070B506460C4621460A4800F02DF905469B
S31508002A50002D01D1401E70BD0648854202D10648A8
S31508002A60051B00E02D1B224629463046FEF77CFF53
S31508002A702046F0E7008000080088000870B5064682
S31508002A800C4621460A4800F00FF90546002D01D1EB
S31508002A90401E70BD0648854202D10648051B00E067
S31508002AA02D1B224629463046FEF75EFF2046F0E7F4
S31508002AB0009000080098000870B505460C462246A6
S31508002AC00249284600F0B1F8204670BD00F4000817
S31508002AD070B505460C4622460249284600F0A5F878
S31508002AE0204670BD0080000810B5044608480069F5
S31508002AF002210843064908610846446100694021E5
S31508002B00084303490861034800F00EF910BD0000A8
S31508002B1000200240FF0F00000C48C068C007C00F25
S31508002B20002801D0012070470848C06804210840E1
S31508002B30002801D00220F6E70448C06810210840A2
S31508002B40002801D00320EEE70420ECE7002002402D
S31508002B50034800698021084301490861704700005D
S31508002B600020024030B504460D460548006901219B
S31508002B7008430349086125800F2000F0D5F830BDC9
S31508002B800020024010B57E2001F0B8FB064800F090
S31508002B900FF87E2001F0B2FB044800F009F87E2009
S31508002BA001F0ACFB10BD000000F40008008000082E
S31508002BB010B5044600F0ACF82046FFF795FFFFF77E
S31508002BC0C7FF10BD70B503460125002208E0500076
S31508002BD01C5A0748844201D0002506E0501C82B2E0
S31508002BE0CE0F761876109642F1DC00BF284670BDE7
S31508002BF0FFFF0000F8B505460E46144600F088F8B3
S31508002C007E2001F07BFB002707E029883046FFF786
S31508002C10A9FFB61CAD1C781C87B2E10F091949102B
S31508002C20B942F2DCFFF794FFF8BDF8B507460C4643
S31508002C3015462946204600F037F80646002E0DD1DF
S31508002C402046FFF7B5FF012080022018FFF7B0FFE6
S31508002C502A4621463846FFF7CDFF24E001208002A8
S31508002C602018401BB0420AD1012080022018FFF725
S31508002C709FFF2A4631463846FFF7BCFF13E001207E
S31508002C80C0022018401BB04208D12046FFF790FF2B
S31508002C902A4631463846FFF7ADFF04E02A46314654
S31508002CA03846FFF7A7FFF8BDF8B505460E462F4686
S31508002CB0E807C00F002801D000BFFEE73146012013
S31508002CC0C002FEF73DFE002901D000BFFEE7002442
S31508002CD00BE020467043471931463846FFF772FF26
S31508002CE0012800D108E0601C84B231460120C002E8
S31508002CF0FEF726FEA042ECDC00BF31460120C002EA
S31508002D00FEF71EFEA04200D100273846F8BD000097
S31508002D1002480349486003484860704723016745ED
S31508002D2000200240AB89EFCD10B5024600BFFFF781
S31508002D30F3FE0346521EFF2400E0641E002CFCD15D
S31508002D40012B01D1002AF2D1064800697721884370
S31508002D50044908613420C860002A01D1052010BD45
S31508002D601846FCE700200240F8B50246CD782F0742
S31508002D703F0FCD7810263540002D01D08D782F4392
S31508002D801446002011E085062B0E0D880126864084
S31508002D903540002D07D025680F269E40B5433E4690
S31508002DA09E4035432560451CE8B20828EBDB141D18
S31508002DB00D882D120095002011E085062B0E0125A1
S31508002DC08540009E3540002D07D025680F269E4079
S31508002DD0B5433E469E4035432560451CE8B2082863
S31508002DE0EBDBCD78282D04D155690E88354355611E
S31508002DF006E0CD78482D03D115690E88354315614F
S31508002E00F8BD70B54D07EB0E082902DA05462035E0
S31508002E1001E0054624352C460F269E402568B54315
S31508002E2016469E403543256070BD000038B50446F9
S31508002E300D460920C006844203D10121480400F04A
S31508002E401DFB1148844203D10121000200F016FB44
S31508002E500E48844203D10121000200F00FFB0C4802
S31508002E60844203D10121080500F008FB684600F0FA
S31508002E701EF868460580012181700021C1706946E7
S31508002E802046FFF771FF38BD0004004800080048D7
S31508002E90000C0048024690680840002801D001202E
S31508002EA070470020FCE741617047016170470021C7
S31508002EB0C9430180022181700421C1707047000056
S31508002EC0F0B58FB00025002600200D900C907E20CE
S31508002ED001F014FA00241AE06100B04A505AFEF7CD
S31508002EE0D8FFAF490790FEF7F9FD0746FFF72CF81C
S31508002EF00022AC4B09910890FEF7E0FE0B910A9070
S31508002F00FFF74AF8A100A84A5050601C84B2042C66
S31508002F10E2DBA5498868FFF717F8A44AA44B059190
S31508002F200490FEF7BDFE0022A24B07910690FEF71D
S31508002F302DFFA14AA14B09910890FEF7B7FE0B9108
S31508002F400A90FFF729F8054697494868FEF7FCFFF7
S31508002F50964A974B05910490FEF7A2FE0022954BE0
S31508002F6007910690FEF712FF934A944B0991089031
S31508002F70FEF79CFE0B910A90FFF70EF806462846C8
S31508002F80FEF7E2FF0022874B05910490FEF78EFEBE
S31508002F900991089029468A48FEF763FD0746FEF719
S31508002FA0D3FF07910690099B089AFEF7EFFE0B914F
S31508002FB00A90FEF7F1FF834908603046FEF7C4FF22
S31508002FC00022784B05910490FEF770FE099108904F
S31508002FD031467B48FEF745FD0746FEF7B5FF0791E4
S31508002FE00690099B089AFEF7D1FE0B910A90FEF708
S31508002FF0D3FF754908607549088BFEF765FF744A63
S31508003000744B03910290FEF759FE0022724B05910C
S315080030100490FEF7BBFE099108906C49088BFEF7F1
S3150800302038FF0746FEF790FF00226B4B0191009090
S31508003030FEF7ACFE0591049062480068FEF784FF2F
S3150800304003910290059B049AFEF72AFE07910690C3
S31508003050099B089AFEF79AFE0B910A90FEF79CFFC9
S315080030600D905A49488BFEF72FFF594A594B039141
S315080030700290FEF723FE0022574B05910490FEF7B7
S3150800308085FE099108905149488BFEF702FF0746CD
S31508003090FEF75AFF0022504B01910090FEF776FE8C
S315080030A00591049048480068FEF74EFF0391029088
S315080030B0059B049AFEF7F4FD07910690099B089A6A
S315080030C0FEF764FE0B910A90FEF766FF0C904348E4
S315080030D00D99FEF76DFC0746FEF704FF40490860A8
S315080030E03E480C99FEF764FC0746FEF7FBFE3D4991
S315080030F008603D48808A3A4909684018C003010CAF
S3150800310039488182C08A374909684018C003010CCA
S315080031103548C1822449C8683449FEF7A2FC0746E7
S31508003120FEF7E0FE81B230488184FF38C138008856
S31508003130FF21F53188422FDD0020244954390880C3
S31508003140194908682A49FEF743FF16D2264820304F
S31508003150407A01280BD124482030C07A002806D1AD
S315080031601A495439486001211F482030C172FF218D
S3150800317001312048FFF799FE0EE01B482030407ABF
S31508003180012804D101021B48FFF78DFE04E0FF2148
S3150800319001311848FFF789FE0FB0F0BD3C01002049
S315080031A000F07F45000008403804002033333333ED
S315080031B03333C33F0000284025068195438BD43F0F
S315080031C00000484354010020580100201402002042
S315080031D0091B9E5E29CB703F00408F400000C84106
S315080031E05C01002060010020800300200000C84226
S315080031F07B142E3F00040048014800687047000011
S31508003200200100200348006803490978401801494D
S3150800321008607047200100202801002008B5012118
S31508003220480400F02BF90121880400F027F96846C4
S31508003230FFF73DFE0121C903684601804821C17098
S3150800324069460920C006FFF78FFD6846FFF72FFE7F
S3150800325001210903684601804821C1706946092091
S31508003260C006FFF781FD6846FFF721FE4021684644
S3150800327001800421C17069460148FFF775FD08BD44
S315080032800004004810B50121C9030920C006FFF74C
S3150800329001FE002839D13E48807B002839D13C48B8
S315080032A0407A01282CD13A482030407A002827D184
S315080032B037482030C079401CC1B235482030C1712A
S315080032C0C07904281CDB04213248FFF7EEFD0021F3
S315080032D02F482030C171AC384089002807D12E48C4
S315080032E02E49486001212A488C38418106E0002091
S315080032F02A494860002126488C38418101F01EF889
S31508003300012123488173817203E0002120488172DC
S315080033108173224880682049884232D900201F4993
S31508003320886000211A4881722030407A002822D10C
S3150800333008211848FFF7B9FD15488C384088032836
S3150800334011DA13488C38408900280CD110482038E7
S31508003350C08A822804DA01210D482030417202E031
S3150800336001210B48C1720A48407A012809D1002078
S315080033700A49486005E000200849486000210448D9
S3150800338041727E2000F0BAFF0148807A10BD000025
S31508003390A003002000040048DC050000C00100204E
S315080033A008B50121480400F069F80121880400F0F5
S315080033B065F86846FFF77BFDFF210E3168460180F8
S315080033C0012181701021C17069461148FFF7CCFCB4
S315080033D0B62168460180012181701021C1706946B5
S315080033E00920C006FFF7C0FC10210920C006FFF718
S315080033F05AFD80210920C006FFF755FD0121044822
S31508003400FFF751FD08210248FFF74FFD08BD0000F0
S31508003410000400488178002925D0174903221202A2
S315080034208918027892109200895802789207D30E6A
S31508003430FF229A40914342789207120E03789B071F
S31508003440DB0E9A4011430C4A03231B02D218037859
S315080034509B109B00D1500178CA06D20E01219140DB
S31508003460054A116007E00178CA06D20E012191408B
S31508003470014A80321160704700E100E0002905D05A
S31508003480054A52690243044B5A6104E0024A5269EA
S315080034908243014B5A61704700100240002905D04B
S315080034A0054AD2690243044BDA6104E0024AD2694A
S315080034B08243014BDA61704700100240002905D0AB
S315080034C0054A92690243044B9A6104E0024A9269EA
S315080034D08243014B9A6170470010024010B500F014
S315080034E031F804494968F02211400909024A515C39
S315080034F0C84010BD00100240EE00002010B5FFF7CE
S31508003500EDFF05494968072212021140090A034AD4
S31508003510515CC84010BD000000100240EE000020BB
S3150800352010B5FFF7DBFF054949680722D2021140AB
S31508003530C90A034A515CC84010BD00000010024089
S31508003540EE000020F8B51E4840680C210840042803
S3150800355002D008282ED101E01A4C2DE01848403038
S315080035600069C007C00F00280AD015484030006916
S3150800357002210840002801D0134802E0114800E063
S31508003580104807460E4840300069FF2109040840E4
S31508003590000C451C0A48403000690721090208400A
S315080035A0000A461C3946694308463146FEF7B2F911
S315080035B0044601E0034C00BF00BF2046F8BD0000EA
S315080035C00010024000127A0000093D0070B504465A
S315080035D000250221074800F00EFC002808D00548FF
S315080035E000F062FC20700221024800F0FCFB012575
S315080035F0284670BD0038014010B500F001F810BD2E
S3150800360000B585B062480068012108436049086032
S3150800361000BF5F480068022108400028F9D05D48CD
S315080036205D4908605D480068102108435B490860E9
S3150800363008460068C008C000086057490968481E5F
S315080036405749FEF767F904905448006804994907F2
S31508003650490F0843514908604D4840685149084098
S315080036604B494860084640689021084348494860E5
S31508003670084640684860484800684649884207D96D
S3150800368043484068052109020843414948600BE060
S31508003690414800684449884206D93D4840680121A6
S315080036A0890208433A4948606B4601AA3A480168C4
S315080036B03E48FEF7C3FF3648403000698008800060
S315080036C033494031086108460069400840000861EE
S315080036D0684600784007400F029068460079400621
S315080036E0400E03902A48C069890508432849C861DD
S315080036F02748403000692E4908402549403108616D
S3150800370003980004029909020843214940310969CE
S3150800371008431F49403108611D4800680121090610
S3150800372008431B49086000E000BF194800680121EA
S31508003730490608400028F7D01548406880088000E8
S315080037401349486008464068022108431049486002
S3150800375000E000BF0E4840680C2108400828F8D150
S315080037600120FFF775F80A48406810218843084980
S3150800377048600120FFF76CF80548406880218843B7
S31508003780034948600120FFF763F805B000BD000053
S315080037900010024000A24A04000100200020024056
S315080037A000366E010FC0FFFF0051250200127A0095
S315080037B0FFF800FF042806D10649096904221143C7
S315080037C0044A116105E00349096904229143014A43
S315080037D01161704700E000E010B5FFF713FD594886
S315080037E00088401C5749088008464068401C4860C5
S315080037F055480068002804D053480068401E5249BE
S3150800380008605248807A012805D14E488068401CD5
S315080038104C49886002E000204A4988604B48C079D4
S31508003820012805D147480069401C4649086102E05D
S315080038300020444908614548007B012805D14148D4
S31508003840C06B401C3F49C86302E000203D49C8637D
S315080038503C4948680A21FEF75DF8002923D13B4810
S315080038602030C1788078814208DD38482030807859
S31508003870401CC1B235482030817014E033482030EE
S31508003880C1788078814200D10DE030482030C17877
S315080038908078814207DA2D4820308078401EC1B2F0
S315080038A02A482030817029482030407A022804D0DE
S315080038B026482030407A032804D12248406B401C11
S315080038C02049486321482030407900280AD11F48FA
S315080038D02030407A042805D11A48406C401C194902
S315080038E0486402E00020174948641848C07B01284C
S315080038F005D11448C06C401C1249C86402E0002077
S315080039001049C8641148007C012805D10D48806C0F
S31508003910401C0C49886402E000200A4988640B4868
S31508003920807904280AD10748006D0949884208D2D7
S315080039300448006D401C0349086502E0002001495F
S31508003940086510BDC00100201C010020A00300204E
S3150800395050C3000010B516480068012108431449F1
S3150800396008600846406813490840114948600846F7
S315080039700068114908400E49086008460068012198
S31508003980890488430A49086008464068C32109042F
S3150800399088430749486008460068084908400449BA
S315080039A008609F2000048860FFF726FE10BD00000F
S315080039B0001002400CC0FFF8FFFFF6FEFFFF8F0065
S315080039C008B501214804FFF759FD02220121092003
S315080039D0C006FFF716FA0221684601801821C17051
S315080039E00121817069460920C006FFF7BDF901214A
S315080039F04804FFF743FD022211460920C006FFF7D7
S31508003A0000FA0421684601801821C17001218170DD
S31508003A1069460920C006FFF7A7F908BD30B587B083
S31508003A2004460D4601210846FFF738FD04A800F0B4
S31508003A3033F90594684605820021018381768174ED
S31508003A4004A90120800700F0F1F8684600F0D2F8D2
S31508003A506021684601700121417000200190002113
S31508003A606846017269460120800700F057F86946E2
S31508003A700120800700F08AF80821C80600F07EF8C1
S31508003A800821C80600F0B0F84021080600F038F80A
S31508003A904021080600F03CF80121880700F00AF8E2
S31508003AA00121880700F01EF80121880700F00EF8AA
S31508003AB007B030BD002904D0026880231A4302608B
S31508003AC003E0026880239A4302607047002904D005
S31508003AD0026801231A43026003E002685208520092
S31508003AE002607047002905D0426C0123DB031A43A4
S31508003AF0426404E0426C0123DB039A434264704744
S31508003B00826907231B039A430B021A438261704793
S31508003B10C26970239A430A43C261704710B5826925
S31508003B2007231B039A430B781B021A4382610A7AFE
S31508003B3012014B781B011A43036A3024A3431A4324
S31508003B4002624A6882630C4A904213D14A7A120189
S31508003B508B781B011A43036AC024A3431A430262E3
S31508003B604A8992008B899B001A4343682401A34320
S31508003B701A43426010BD0000002C014082690123EF
S31508003B80DB029A430B021A438261704710B5C26979
S31508003B9070239A430B781A43C2610A7A12024B7849
S31508003BA01B021A43036A03242402A3431A4302622C
S31508003BB04A68C2630B4A904213D14A7A12028B783A
S31508003BC01B021A43036AA400A3431A4302624A89E2
S31508003BD012018B891B011A434368A400A3431A43A5
S31508003BE0426010BD002C0140C26908239A430A436B
S31508003BF0C261704700210170417081704160017295
S31508003C00417241818181704701229207904201D118
S31508003C10816301E08AB2826370470122920790426B
S31508003C2001D1C16301E08AB2C26370470268032307
S31508003C301B029A430B891A430260134A904206D024
S31508003C4001229207904202D0104A904205D102689A
S31508003C5070239A438B781A4302600B4A904205D028
S31508003C600B4A904202D00B4A904205D1026B120AC7
S31508003C7012028B7A1A4302634A68C2620A8882620F
S31508003C800122426170470000002C014000040040F8
S31508003C9000440140004801400021C9434160002119
S31508003CA00180018181708172704710B5FFF7A4FA0F
S31508003CB010BD000070B5FFF711FC05467D21C9004F
S31508003CC0FDF728FE0446601E0C49884200D90CE020
S31508003CD0601E0B4948610321081F00F085FB002080
S31508003CE0074988610720086100BF0420FFF762FDC5
S31508003CF00021481E00F078FB70BD0000FFFFFF00A2
S31508003D0000E000E010B50221154800F07DF8002813
S31508003D1024D0134800F0C8F8C4B21248C079002865
S31508003D2003D1204600F06EFF14E00E48C079022841
S31508003D3010D10C48007A00280CD10B488079AA28A3
S31508003D4004D10948C471012106480172AA2C01D17F
S31508003D50054884710221024800F045F810BD0000AC
S31508003D6000380140A0030020F804002010B50446DE
S31508003D702146054800F09CF800BF0121024800F0E2
S31508003D803AF80028F9D010BD0038014070B505464C
S31508003D900E4600247E2000F0B1FA00BF20E0042C75
S31508003DA019DD701EA04216DD285D7E2806D17D200D
S31508003DB0FFF7DCFF5E20FFF7D9FF0FE0285D7D28BF
S31508003DC005D1FFF7D3FF5D20FFF7D0FF06E0285D9A
S31508003DD0FFF7CCFF02E0285DFFF7C8FF601C84B23E
S31508003DE0B442DCDB70BD41617047826952085200FB
S31508003DF00A4382617047024690680840002801D04D
S31508003E00012070470020FCE70246D06808400028D9
S31508003E1001D0012070470020FCE7002A03D003697F
S31508003E200B43036102E003698B430361704700009B
S31508003E3070B504460D460026E06930218843297985
S31508003E400843E061E06944218843A9790843E061B1
S31508003E50E06980088000297A0843E061A069182192
S31508003E60884369890843A061A06904218843297B9E
S31508003E700843A0610B48844203D1FFF751FB06466D
S31508003E8002E0FFF73BFB064630462968FDF742FD90
S31508003E900009206230462968FDF73CFD0007000F3F
S31508003EA0606270BD0038014001464868C0B270477C
S31508003EB0CAB2026070474B21C90101603021017105
S31508003EC00021817101721821418100210173704717
S31508003ED010B51C484088030000F077FA0504111E47
S31508003EE0292A2B0017486C30808CFF211B31884209
S31508003EF004DA01211348418000F020FA19E011483C
S31508003F006C30808CFF210531884204DA02210D4885
S31508003F10418000F013FA0CE00A486C30808CFD28CA
S31508003F2004DA03210748418000F008FA01E000E0BE
S31508003F3000BF00BF03488C30407A002801D100F04A
S31508003F40FDF910BD1403002010B53048408800283C
S31508003F5006D0012813D0022820D0032854D12CE0FB
S31508003F6080210920C006FEF7A0FF01212848FEF798
S31508003F709CFF10210920C006FEF797FF44E00121A7
S31508003F802348FEF792FF80210920C006FEF78BFF23
S31508003F9010210920C006FEF786FF35E0802109209A
S31508003FA0C006FEF782FF01211948FEF77CFF1021A3
S31508003FB00920C006FEF777FF26E016494868CD2196
S31508003FC0FDF7A8FCC007C00F002805D080210920EE
S31508003FD0C006FEF768FF0DE00E494868CD21FDF7DB
S31508003FE099FCC007C00F002804D180210920C0060B
S31508003FF0FEF75BFF01210648FEF755FF1021092051
S31508004000C006FEF750FF00BF00BF10BD1403002016
S3150800401000040048C001002010B5A04880790300BC
S3150800402000F0D3F90504336CAFFDFC009B4820383B
S31508004030808CFF210531884202DB01219748817176
S3150800404040219748FEF726FF00281DD09549486865
S31508004050FF21F531FDF75EFCC007C00F002805D12A
S3150800406080210920C006FEF71EFF04E080210920F2
S31508004070C006FEF71AFF10210920C006FEF713FF37
S3150800408001218748FEF70FFF06E184482038808C17
S31508004090FF211B31884202DB0221804881714021C1
S315080040A07F48FEF7F7FE002827D07E494868FF219B
S315080040B0F531FDF72FFCC007C00F002804D10121F8
S315080040C07748FEF7F0FE03E001217548FEF7EDFE9E
S315080040D080210920C006FEF7E6FE10210920C00649
S315080040E0FEF7E1FE6D488C384088012805D001218D
S315080040F06A488C38418000F021F9CDE067482038BD
S31508004100808CFF212531884202DD032163488171B5
S3150800411040216348FEF7BEFE002831D06149486851
S31508004120FF21F531FDF7F6FBC007C00F00280ED1B9
S3150800413080210920C006FEF7B8FE01215848FEF77F
S31508004140B4FE10210920C006FEF7AFFE0DE080215F
S315080041500920C006FEF7A7FE10210920C006FEF7B3
S31508004160A2FE01214E48FEF79EFE4C488C38408838
S31508004170002805D0002149488C38418000F0DEF837
S315080041808AE040214648FEF785FE00284ED00121E8
S3150800419009030920C006FEF77DFE002811D08021FC
S315080041A00920C006FEF781FE01213D48FEF77DFE87
S315080041B010210920C006FEF778FE042137488171D0
S315080041C026E038494868FF21F531FDF7A3FBC0070B
S315080041D0C00F00280ED180210920C006FEF765FE13
S315080041E001212F48FEF761FE10210920C006FEF7BF
S315080041F05CFE0DE080210920C006FEF754FE102162
S315080042000920C006FEF74FFE01212548FEF74BFEA2
S3150800421022488C384088002808D001E03BE006E0B8
S3150800422000211E488C38418000F088F834E040218F
S315080042301B48FEF72FFE00282CD018488C384088DB
S31508004240002805D0002115488C38418000F076F802
S315080042501448006D144988420ED280210920C006F0
S31508004260FEF723FE01210E48FEF71FFE1021092046
S31508004270C006FEF71AFE0DE080210920C006FEF7EB
S3150800428012FE10210920C006FEF70DFE0121044882
S31508004290FEF709FE00E000BF00BF10BDA003002026
S315080042A000040048C00100203075000003488068FB
S315080042B0400840000149886070470000002C004013
S315080042C080210143014A116070470000002C00401C
S315080042D003488068002801D0012070470020FCE7C9
S315080042E0002C004010B5FFF7F3FF002804D0FFF7B5
S315080042F0DDFF662000F002F810BD00004106490EF9
S31508004300014A116070470000002C004004494968C2
S31508004310FF22813291430143014A516070470000F0
S31508004320002C004004494968C909C9014206520ED1
S315080043301143014A51607047002C004010B57E2099
S31508004340FFF7DCFF0948FEF733FC09490948818273
S315080043500621143000F09AF8064914318881402263
S31508004360024904481430FEF760FC10BD00900008AE
S31508004370FBAA00000003002070B505460C46012183
S31508004380C802FFF78BF8FF208130FFF7BFFF2046F2
S31508004390FFF7C8FF2846FFF793FF70BD2021020CE0
S315080043A001D010211046020A01D010460839020928
S315080043B001D01046091F820801D01046891E4208FE
S315080043C001D0881E7047081A704730B47446641EB8
S315080043D02578641CAB4204D3635D5B00E31830BCEC
S315080043E018471D46F8E7000010B5002819DB1A4AD9
S315080043F003231B02D21883089B00D2588307DC0EBE
S31508004400FF23A3409A438B071B0E8407E40EA340A1
S315080044101A43114B032424021B198408A4001A51B9
S3150800442018E00E4A03071B0F083B9B089B00D2584F
S315080044308307DC0EFF23A3409A438B071B0E8407D2
S31508004440E40EA3401A43054B0407240F083CA408AE
S31508004450A4001A5110BD000000E100E01CED00E0C8
S3150800446002E008C8121F08C1002AFAD1704770472F
S31508004470002001E001C1121F002AFBD1704700008D
S315080044800149086070470000BC01002010B50246CB
S315080044900023002901D1002010BD03E01488921CD6
S315080044A0E01883B208464C1EA1B20028F6D1184679
S315080044B0F2E70000F8B50027002600240025FC488E
S315080044C0007A01286FD17E20FFF718FFF948C079D6
S315080044D00002F849097A08430746F648467A847A74
S315080044E00246D17A107B00F0CBFC05460021F04845
S315080044F00172F149781A8F426FD01EDCEF49781A9B
S315080045008F426BD010DCEE49781A8F4267D006DCF2
S31508004510442F1CD0EB483818002872D1E4E18828CB
S3150800452070D08928F9D174E101286CD002286BD0A3
S3150800453003286AD00428F0D135E10300FFF745FFC8
S315080045400C61C0FAF861611926768E415C61062E07
S3150800455009D1DD48007800280AD100F03FFF012084
S31508004560D949087004E0152E02D1012000F036FF63
S31508004570D5E1CF482030407A002806D0CC482038EC
S31508004580828AC18A002000F083FEC8E1002C0BD184
S31508004590C7482038C08A00231A46F0210090FE201A
S315080045A000F0ABFE0CE0BBE1012C09D1C048203875
S315080045B0808A01230022F0210090FE2000F09DFE53
S315080045C0ADE1002C0CD1C148408800231A46F321DE
S315080045D00090FE2000F091FE0DE05AE05BE18EE1CE
S315080045E0012C08D1B948808901230022F3210090C3
S315080045F0FE2000F082FE92E1002C07D1B3484580E8
S3150800460006E08BE119E122E16AE07AE0AF488581AC
S31508004610AE488089FF21F531884206DA00F0D0FAE3
S315080046200022FE21F42000F09CFE78E1002C09D13E
S31508004630A648808800231A46F1210090FE2000F043
S315080046405CFE0AE0012C08D1A048C089012300229B
S31508004650F1210090FE2000F050FE60E1002C02D10E
S315080046609A48858003E0012C01D19848C58197486E
S315080046708088FF21F53188420ADC9448C08988423F
S3150800468006DC00F09DFA0022FE21F22000F069FE09
S3150800469045E1002C09D18D48C08800231A46E92136
S315080046A00090FE2000F029FE09E0012C07D1192010
S315080046B001230022E9210090FE2000F01EFE2EE1D3
S315080046C0002C01D18148C580FF202D30854206DAAD
S315080046D000F076FA0022FE21EA2000F042FE1EE1F2
S315080046E0002C0CD1794800896421484380B2002304
S315080046F01A46E2210090FE2000F0FFFD00E000BF10
S315080047000DE1002C06D164212846FDF719F981B27E
S315080047106E4801816D480089FF21F531884206DC23
S3150800472000F04EFA0022FE21E32000F01AFEF6E021
S315080047301EE0FFE7002C0CD16448408964214843F9
S3150800474080B200231A46EB210090FE2000F0D5FD2A
S315080047500DE0012C0BD15D48008A6421484380B2E4
S3150800476001230022EB210090FE2000F0C6FDD6E0D2
S31508004770002C07D164212846FDF7E2F881B2534898
S31508004780418108E0012C06D164212846FDF7D8F8B6
S3150800479081B24E48018200F013FA0022FE21EC2075
S315080047A000F0DFFDBBE0012C1AD141488C38408867
S315080047B003280CDA3E488C384089002807D10121A5
S315080047C03B48203041720020404954394860002255
S315080047D0FE21E42000F0C5FD01213548417217E0AD
S315080047E0002C10D10021324841722030417200223B
S315080047F0FE21E42000F0B5FD002033490870334956
S315080048005439486004E00022FE21E42000F0A9FDA6
S3150800481085E0002C0FD12748C07A32280CDC2548C1
S31508004820C17A2A48418200F0CBF90022FE21DF2016
S3150800483000F097FD00E000BF71E02448408A00239D
S315080048401A46DE210090FE2000F057FD67E0002C96
S315080048500FD11848C07A32281CDC1648C17A1B4882
S31508004860818200F0ADF90022FE21E12000F079FDF9
S3150800487010E0012C0ED10F48C07A32280ADC0D4808
S31508004880C17A1248C18200F09BF90022FE21E1207C
S3150800489000F067FD43E0002C1AD10C48808A0023FB
S315080048A01A46E0210090FE2000F027FD1BE00000DC
S315080048B0A0030020F8040020E9FE0000E0FE000046
S315080048C056FE0000AB01FFFFB801002014020020CD
S315080048D0012C08D11348C08A01230022E021009048
S315080048E0FE2000F00AFD1AE0002C07D101210E482F
S315080048F0C171002202210D48FFF78FFA0FE0002C44
S315080049000BD1FF2101310A48FDF747F80020084975
S31508004910891F088002210448C17100E000BF00BF5A
S31508004920F8BD000014020020A00300200038014052
S31508004930FE040020F0B589B0002008900790069084
S315080049403848007A01286BD137488079AA2864D17B
S315080049503548C079322860DA3348C07900285CDDEA
S315080049603149C97908461938FDF788FA0890089830
S31508004970FDF7EAFA04462D4A2D4BFDF79FF900226A
S315080049802C4B01910090FDF7E7F8039102902A4815
S315080049900068FDF7D9FA0646039B029AFDF7F6F971
S315080049A005910490FDF7F8FA079024490798FDF752
S315080049B058F80446FDF796FA81B22148018308980B
S315080049C0FDF7C2FA0646194A194BFDF777F9044668
S315080049D00022184BFDF7C0F80391029019480068A9
S315080049E0FDF7B2FA01910090039B029AFDF7CEF902
S315080049F005910490FDF7D0FA069010490698FDF740
S31508004A0030F80446FDF76EFA81B20D48418300F08E
S31508004A10D7F800210348C17141720021014801728B
S31508004A2009B0F0BDA0030020F8040020091B9E5E13
S31508004A3029CB703F0000F03F5401002000007A4463
S31508004A40140200205801002070B505460E4614468B
S31508004A50002E02D0012E4AD120E0002D02D0012DD1
S31508004A601AD10CE0602101208007FFF749F80021E0
S31508004A7001208007FFF7C8F81E4804700CE0602183
S31508004A8001208007FFF744F8002101208007FFF77F
S31508004A90C4F81948047000BF00BF28E0002D02D0F2
S31508004AA0012D22D110E013480078A0420BD06021D6
S31508004AB001208007FFF724F8214601208007FFF729
S31508004AC0A3F80C48047010E00B480078A0420BD0FD
S31508004AD0602101208007FFF71BF821460120800787
S31508004AE0FFF79BF80448047000BF00BF00BF00BF73
S31508004AF070BD00006A0100206B01002010B5052476
S31508004B0021E080212C48FCF748FF80212A48FDF740
S31508004B1079FF0F212848FFF7B9FC2749C98B884236
S31508004B200CD125481438808A2449884204D000F0DC
S31508004B30CFF900F045F800E010BD04E0002000E0E1
S31508004B40401C8028FCDB2046611ECCB20028D8D148
S31508004B5000BF052423E080211748FCF71EFF8021AB
S31508004B601548FDF76DFF0F211348FFF78FFC124913
S31508004B70C98B88420ED110481438808A0F4988425A
S31508004B8004D000F0A5F900F01BF802E000F018F8D0
S31508004B90D2E704E0002000E0401C8028FCDB204629
S31508004BA0611ECCB20028D6D100BF00F091F900F002
S31508004BB007F800BFC0E7000014020020FBAA0000A7
S31508004BC010B57E20FFF79AFBFDF7DCFF0B490C4872
S31508004BD081820F211430FFF759FC09491431C88323
S31508004BE0802107481430FDF767FF7E20FFF786FB14
S31508004BF0802103481430FDF76BFF10BDFBAA0000A7
S31508004C000002002070B5044600257E20FFF776FBDB
S31508004C1098480088FA280ADD0020964908809649AF
S31508004C200870FF2101319348801DFCF7B6FE9248B3
S31508004C3000780300FFF7C9FB08052031425BD5EC75
S31508004C40FDFC7E2C11D100208A49088001208A4962
S31508004C500870884801880088401C864A1080901D84
S31508004C60445400201146C87002E00020814908809B
S31508004C70002080490871FBE07E4801880088401CB6
S31508004C807C4A1080901D445402207B4908701046C7
S31508004C900079001911460871EAE07648018800880B
S31508004CA0401C744A1080901D4454032072490870B1
S31508004CB010460079001911460871D9E06D48018837
S31508004CC00088401C6B4A1080901D445404206A4991
S31508004CD00870104600790019114608710846C47014
S31508004CE0C078002802D1052063490870C0E06148F1
S31508004CF04079012856D15E2C1CD15E4800797E3059
S31508004D005C4908717E215B4802880088401C594B23
S31508004D101880981D8154801FC078401EC0B219465D
S31508004D20C870002802DC0520534908700020514944
S31508004D30487155E05D2C1CD14E4800797D304D49AF
S31508004D4008717D214B4802880088401C494B188011
S31508004D50981D8154801FC078401EC0B21946C8707D
S31508004D60002802DC052044490870002041494871A2
S31508004D7036E04048007900193E490871084601881E
S31508004D800088401C3B4A1080901D4454801FC07800
S31508004D90401EC0B21146C870002821DC05203649DD
S31508004DA008701DE07D2C03D101203249487117E0B7
S31508004DB03048007900192F4908710846018800888B
S31508004DC0401C2C4A1080901D4454801FC078401EF9
S31508004DD0C0B21146C870002802DC052026490870B2
S31508004DE046E024480079C043401CC5B2A54203D119
S31508004DF006202149087002E007201F4908701D484F
S31508004E0001880088401C1B4A1080901D44542FE0DE
S31508004E10184801880088401C164A1080901D445482
S31508004E207E2C0BD10121154801720020114601E0A4
S31508004E301DE00DE008801049087008E000200D49C3
S31508004E40088000210D48017200200B4908700FE008
S31508004E50002009490870074801880088401C054A4F
S31508004E601080901D445400201146088000E000BFC1
S31508004E7000BF70BDF8040020B7010020A003002081
S31508004E8070B50246002013460C461D02FF26360260
S31508004E9035402543284670BD00BF00BF00BF00BF90
S31508004EA000BF00BF00BF00BF00BFFEE706490748B6
S31508004EB081820021143041805F218180C180018177
S31508004EC00021418170470000FBAA00000003002072
S31508004ED000B5134913488182FF21143041800F2100
S31508004EE00181A021C180D22181801E214181AF216B
S31508004EF0C1818C210182BE2181810B4901830A4926
S31508004F0023314183052141820A218182C182002100
S31508004F1081830F21FFF7BAFA02491431C88300BD0D
S31508004F20FBAA0000000200205A25000010B57E20CA
S31508004F30FFF7E4F95948C07A01282AD15748407A38
S31508004F4001281CD156494868C821FCF7E3FCC0076C
S31508004F50C00F002805D180210920C006FDF7A3FF50
S31508004F600DE04F494868C821FCF7D4FCC007C00FBC
S31508004F70002804D080210920C006FDF796FF1021DD
S31508004F800920C006FDF78FFF01214648FDF78BFF74
S31508004F9010BD4248407A01287DD140482030407AE9
S31508004FA0002802D0012839D110E040213D48FDF7FC
S31508004FB071FF002807D13A48006D3B49884204D260
S31508004FC0FEF7C2FF01E0FFF727F863E034494868B7
S31508004FD0FF21F531FCF79EFCC007C00F00280ED153
S31508004FE080210920C006FDF760FF01212D48FDF745
S31508004FF05CFF10210920C006FDF757FF0DE0802150
S315080050000920C006FDF74FFF10210920C006FDF74D
S315080050104AFF01212348FDF746FF3BE01F482030A1
S31508005020407A052827D11E494868FF21F531FCF743
S3150800503071FCC007C00F00280ED180210920C006C8
S31508005040FDF733FF01211748FDF72FFF102109202F
S31508005050C006FDF72AFF1CE080210920C006FDF7DF
S3150800506022FF10210920C006FDF71DFF01210D486A
S31508005070FDF719FF0DE080210920C006FDF715FF91
S3150800508001210848FDF711FF10210920C006FDF788
S315080050900CFF00BF00BF00BF7AE70000A003002096
S315080050A0C00100200004004830750000FEF752FCDD
S315080050B0FEF776F9FDF7FEFBFDF79AF90B20FDF7EB
S315080050C0C9F80C20FDF7C6F80920FDF7C3F8032038
S315080050D0FDF7C0F801215648FDF730FA4B200002CB
S315080050E0FDF752FBFEF79AF8FEF76AFC1A216320D1
S315080050F0FEF794FC01214F4841720021C172FFF767
S31508005100FDFCFEF7D7FD00F09DF8FEF71DFF7F2199
S315080051107E20FFF731F98AE04648C07900280AD18F
S31508005120FDF734FAFFF702FFFFF7C4F9FEF7AAF80E
S3150800513000F086FF78E03F48C079012836D1002381
S3150800514001221946184600F0A9F900231A461946FD
S31508005150184600F0A3F9384840683849884204D907
S3150800516008213748FDF79FFE1DE033494868FF21AF
S31508005170F531FCF7CFFBC007C00F00280ED1802100
S315080051800920C006FDF78FFE10210920C006FDF78D
S315080051908AFE01212A48FDF786FE04E0102109202F
S315080051A0C006FDF782FEFDF79BFA3DE02148C0796F
S315080051B0022839D1FDF7EAF9FEF764F8002301223F
S315080051C01946184600F06AF900231A461946184681
S315080051D000F064F9184840681849884204D908213B
S315080051E01748FDF760FE1DE013494868FF21F531B1
S315080051F0FCF790FBC007C00F00280ED180210920BC
S31508005200C006FDF750FE10210920C006FDF74BFE2B
S3150800521001210B48FDF747FE04E010210920C006CE
S31508005220FDF743FEFFF786FB7E20FFF767F873E777
S3150800523000240140A0030020C0010020204E0000E9
S315080052400004004810B540210F48FCF7A6FB402192
S315080052500D48FDF713FC06210B48FFF717F90A4915
S31508005260898988420AD108481438808A07498842B9
S3150800527008D0FFF71BFEFFF761F803E0FFF716FEFD
S31508005280FFF75CF810BD000014030020FBAA00001D
S31508005290F7B5A0B00C46154680216846FCF77DFB9D
S315080052A0002700267E2168460170FE214170EF2105
S315080052B081700721C17020990171002141718471A3
S315080052C02112C171012101724572291281720126CA
S315080052D005E06846805DC019C7B2701CC6B20B2EC1
S315080052E0F7DBF843401CC1B26846C1727E210173E0
S315080052F00D21FEF74BFD23B0F0BDFFB585B0054681
S315080053000E460E9F00200190029003900490009094
S3150800531000247E2168460171457186710421C17198
S31508005320079901720899417287723912C17201246C
S3150800533007E001A8015D00980818C0B20090601C3B
S31508005340C4B2082CF5DB0098C043401CC1B26846BD
S3150800535001737E2141730A2101A8FEF717FD09B0E2
S31508005360F0BDF7B584B005460E46002000900190C2
S3150800537002900390002700247E216846017046703B
S3150800538085700121C170694606980871012405E0F7
S315080053906846005DC019C7B2601CC4B2052CF7DBAD
S315080053A0F843401CC1B2684641717E2181710721CC
S315080053B0FEF7ECFC07B0F0BD70B504460D467E203E
S315080053C0FEF79CFF03E02078641CFEF7CFFC284616
S315080053D0691E8DB20028F6D170BD000030B5A1B0A7
S315080053E00446802101A8FCF7D8FA0025002C02D033
S315080053F0012C20D10FE07E21684601710021417100
S31508005400442181711321C1711522104902A8FCF7A4
S31508005410ABFA192510E07E2168460171FE2141711B
S31508005420442181713321C1713622094902A8FCF74A
S315080054309BFA3A2500E000BF00BF802D03DA294613
S3150800544001A8FFF7B9FF21B030BD00006C010020AC
S3150800545081010020F8B506460C46FCF797FE051EA6
S315080054600F4600D00120014349000B484908411A5C
S31508005470C90F0DD0002E01D0012100E000210C43F8
S3150800548061004908401AC00F02D10120FEF7F8FF53
S3150800549028463946F8BD00000000F07FFFB58DB0FC
S315080054A005460E46174600200B9000240A900990E0
S315080054B00890FE480078642803D0FD48C078642820
S315080054C004D10121FA482038017303E00021F84885
S315080054D020380173002F02D0012F7BD130E2F54826
S315080054E0C089B04202D1F348C48A00E00524052CDD
S315080054F001DC052402E0322C00DB0524301BA8421F
S315080055000FDDEB482038C07B00284CD1E9485438D9
S315080055104068E849543988610121E5482038C17353
S3150800552041E03019A8423EDCE1482038C07B01281A
S3150800553039D1DF48407901282FD1DE4854384068F0
S31508005540DC4954398969401ADB4988420DD2D84862
S31508005550AC380089462820DDD548AC380089801E3D
S3150800556081B2D348AC38018117E0D2485438406834
S31508005570D04954398969401A7D21890188420CD954
S31508005580CB48AC3800895F2807DAC948AC380089A7
S31508005590801C81B2C648AC3801810121C4484171DA
S315080055A000212038C173C2482038C07B012878D131
S315080055B0301BA84276DDBF48543840687D21C900B3
S315080055C0884208D26420B94908700021B8482038B2
S315080055D08174AEE1FEE3B6482038807C00286AD1A3
S315080055E00121B34820388174B248808964285ADA80
S315080055F0AF484038818AC08B081A81B2AC48403817
S3150800560001840146088CFCF744FC01460690AB4829
S315080056100068FCF763FA0790FCF796FCA84A03C2F1
S31508005620A3494039898C49430846FCF739FC079158
S315080056300690A3480CC80698FCF740FBA04A03C28C
S315080056409F4903C9FFF706FF07910690FCF7A4FCDC
S315080056509C49086096494039888CFCF71AFC014633
S31508005660059098480068FCF739FA97490690FCF7C0
S31508005670F8F90790FCF736FC944908700846007854
S3150800568064280ADC8D480068FCF75EFC0022904B13
S3150800569007910690FCF76CFC08D864208B490870C3
S315080056A004E043E15BE0642088490870804840389C
S315080056B0818A41873DE17F485438406C7D21C90085
S315080056C0884247D900207B49543948647F48007886
S315080056D064283BDA76484038818A408F814230DD3B
S315080056E00121890775480068FCF762F90790FCF7FD
S315080056F0F9FB81B26E484038828A408F101A81427F
S3150800570005DA72480078801E704908701EE06849FC
S3150800571040398A8A498F501AFCF7B0FB07906748C8
S3150800572001680798FCF754FC10D268480078801C7A
S315080057306649087008460078642807DD6420087002
S3150800574004E062480078401D6049087058484038AF
S31508005750818A41875D48007854490870E9E05448D1
S315080057604079002870D153488089642803DB642077
S315080057704E490870DDE04F48543840687D21C9001D
S31508005780884207D2642049490870002148482038D1
S315080057908174CEE046482038807C00285DD10121FE
S315080057A04348203881744348808964284DDA404844
S315080057B04038818AC08B081A81B23D484038018436
S315080057C00146088CFCF765FB014606903B480068D5
S315080057D0FCF784F90790FCF7B7FB394A03C234494A
S315080057E04039898C49430846FCF75AFB07910690CD
S315080057F033480CC80698FCF761FA314A03C23049A7
S3150800580003C9FFF727FE07910690FCF7C5FB2D494C
S31508005810086027494039888CFCF73BFB0146059010
S3150800582028480068FCF75AF927490690FCF719F941
S315080058300790FCF757FB2549087008460078642846
S3150800584006DD6420087003E06AE064201F490870DA
S3150800585017484038818A41876BE016485438406CAF
S315080058607D21C900884256D9002012495439486416
S315080058700F484038818A408F814244DD01218907DB
S315080058800E480068FCF794F80790FCF72BFB81B2EA
S3150800589007484038828A408F101A81421ADA0B4824
S315080058A00078801E0949087032E00000EA000020EE
S315080058B0C00300201402002070170000CC0000204E
S315080058C0D0000020D80000200000C842E9000020CF
S315080058D00000F03FFE498A8A498F501AFCF7CEFA33
S315080058E00790FC4801680798FCF772FB10D2FA4843
S315080058F00078801CF849087008460078642807DD97
S315080059006420087004E0F4480078401DF2490870E5
S31508005910EF48818A4187F0480078F049087008E026
S31508005920EB486C38007AED49087002E00020EB4934
S315080059300870EA48027838461099FFF785F86EE34A
S31508005940E3484030407A012804D002287DD0032855
S315080059507CD196E0E2484088B04202D1E048448AC9
S3150800596000E00A24DE484188408A081AA84209DB72
S31508005970DB4854384068DA49543988620020D949E6
S3150800598008701AE0D6484088A84216DCD548007840
S31508005990002812D1CE48818C81870120D149087010
S315080059A0CF4854384068CE495439896A401ACC4998
S315080059B054390862084640680863C9488188808A5D
S315080059C0081AA84209DB0020C7490870C448543899
S315080059D04068C3495439C86217E0C1488088A8425C
S315080059E013DCC148007800280FD1B948818CC187DB
S315080059F00120BD490870BA4854384068B849543936
S31508005A00C96A401AB64954394862B5485438406894
S31508005A107D21C90088422AD3AD482030407C002821
S31508005A2025D1AB48818C4030018001212038417452
S31508005A30014620310888FCF72CFA01460590AB4848
S31508005A40FCF74CF8AA49069001E011E022E0FCF7C1
S31508005A5008F80790FCF746FAC1B29D484030017134
S31508005A600079642803DB64219948403001711AE003
S31508005A709B484088B04202D19948448A00E00A24EB
S31508005A8011E097488088B04202D19548848A00E0A0
S31508005A900A2408E092488088B04202D19048848A55
S31508005AA000E00A2400BF00BF052C01DC052402E043
S31508005AB0322C00DB3224301BA8421ADB88485438C3
S31508005AC0406887495439C86100204863886380481C
S31508005AD045842030007C002806D11E217C484030B1
S31508005AE081700121203801740021794820304173E2
S31508005AF012E13019A84211DC75482030007C0128D3
S31508005B00F6D10021724820300174FF38E138406828
S31508005B1073495439C86100204863FDE0B542E7DBA4
S31508005B206B484030407A0128E2D169484030807994
S31508005B300028DDD16A48408A0A280BDB68495439AF
S31508005B40086AFCF7A6F96B490790FBF7C7FF6A498D
S31508005B5008601EE06248408A0A280FDA6048408AD0
S31508005B6007280BDD5E495439086AFCF792F9634940
S31508005B700790FBF7B3FF604908600AE058495439B3
S31508005B80086AFCF786F95E490790FBF7A7FF5A49AA
S31508005B9008604F49888FFCF77CF94D490690888F35
S31508005BA0FCF777F90490544801680498FBF759FF05
S31508005BB005900699FBF755FF0790FCF7C5F9514A7A
S31508005BC003C24349888FFCF77FF9039102904D4938
S31508005BD003C9FFF73FFC01910090039B029AFCF76B
S31508005BE0D5F80022484B05910490FCF767F8079111
S31508005BF00690FCF78BF981B235486C3881803849B4
S31508005C005439486AFCF745F93C490790FBF766FFA3
S31508005C10394908602E49C88FFCF73BF92C4906908C
S31508005C20C88FFCF736F90490334801680498FBF7E7
S31508005C3018FF05900699FBF714FF0790FCF784F9FF
S31508005C40304A03C22249C88FFCF73EF903910290F5
S31508005C502C4903C9FFF7FEFB01910090039B029AAA
S31508005C60FCF794F80022284B05910490FCF726F8D7
S31508005C7007910690FCF74AF981B215486C38C1803D
S31508005C8017488089642844DA15498889FCF701F998
S31508005C90134954390690086BFCF7FBF81B49029028
S31508005CA0FBF71CFF0E4904904A880949898B501A4C
S31508005CB0FCF7E4F803900499FBF710FF05900699A2
S31508005CC0FBF7CFFE0A490790FBF708FF01491FE0DB
S31508005CD080030020CC000020E9000020EA00002014
S31508005CE014020020DC000020DD00002000008243B2
S31508005CF00000C84200803B45C40000200000FA446A
S31508005D000080BB44E00000200000594000007A44AF
S31508005D1008600121C4488171C3482038007C0028E6
S31508005D207CD001287BD1C0488078C0490978884250
S31508005D3008DA0021BC488170203801740020BC496B
S31508005D4088641CE1301BA84210DDB7482038407C27
S31508005D50012803D1B4480179C17002E06421B24830
S31508005D60C1700121B0482038017308E1AE48407A75
S31508005D70012804D0022813D003287DD188E03019E1
S31508005D80401BA04208DA3019401B201A5F21081A66
S31508005D90C1B2A548C17002E05F21A348C170EDE019
S31508005DA0A348406BA249896B401A7D21C9008842E5
S31508005DB04BD99F48406B9E4988639B484038408C26
S31508005DC0A84211DD9848AC3880880A3081B29648D6
S31508005DD0AC3800E023E18180C088642832DB642186
S31508005DE09148AC38C1802DE08F494039498C691AF1
S31508005DF0E20F12195210521C914211DA8A48AC3835
S31508005E008088801C81B28848AC388180C088642824
S31508005E1018DB64218448AC38C18013E0B0E0E7E0C1
S31508005E2081494039498C691AE20F12195210921C9D
S31508005E30914207DD7C48AC388088801E81B27A485A
S31508005E40AC38818078484038458479484068784934
S31508005E50C969401A7749884214DD7348AC38808886
S31508005E60401D81B27048AC3881808088642805DB83
S31508005E7064216D48AC3800E07CE081806C4840685D
S31508005E806B49C8616848AC380179AC30C17075E0B7
S31508005E906748406B6649896B401A7D21C90088426C
S31508005EA047D96348406B624988635F484038408CED
S31508005EB0A8420FDD5C48AC38C0880A3081B25A481F
S31508005EC0AC38C180C088642830DB64215648AC38B9
S31508005ED0C1802BE054494039498C691AE20F1219DE
S31508005EE05210521C91420FDA4F48AC38C088801CB9
S31508005EF081B24D48AC38C180C088642816DB64215D
S31508005F004948AC38C18011E047494039498C691A7B
S31508005F10E20F12195210921C914207DD4248AC3822
S31508005F20C088801E81B24048AC38C1803E4840389F
S31508005F3045843F4840683E49C969401A3E498842F7
S31508005F4012DD3948AC38C088401D81B23648AC38B5
S31508005F50C180C088642803DB64213348AC38C1801B
S31508005F60334840683249C8612F48AC388179AC302B
S31508005F70C17003E032212C48C17000BF00BF3BE06E
S31508005F802948407A012823D13019A8421CDB264823
S31508005F90AC380179AC30C1703019801EA8420FDDCB
S31508005FA026480078002822D11F48AC388088401D32
S31508005FB081B21D48AC38818001202049087016E05E
S31508005FC000201E49087012E000211748C1700EE033
S31508005FD01548407A042803D01348407A052803D187
S31508005FE000211148C17002E00A210F48C17003E080
S31508005FF000210D48C17000BF00BF0B48407A012838
S3150800600006D10948C27838461099FEF71DFD05E005
S315080060100548827838461099FEF716FD00BF00BF7E
S315080060200B9811B0F0BD0000C0030020EA00002064
S31508006030C001002088130000581B0000E80000205B
S3150800604010B5F748407A002876D0F5484038C08A17
S31508006050FF217D31884204DCF1484038808A884235
S315080060600ADDEF482038C07A002805D1ED49486096
S315080060700121EB482038C172EA48C06BEA498842D8
S315080060800AD9E7482038C07A002805D1E54948608A
S315080060900121E3482038C172E1482038C07B012835
S315080060A01ED1E048C06CE14988421DD90020DD496F
S315080060B0C864DB484038418B808A81420BDBD8486C
S315080060C02038C07A00280FD1D64948600121D44823
S315080060D02038C17208E0D2484038818A418303E0FB
S315080060E0CF484038818A4183CD482038007C012832
S315080060F01ED1CC48806CCD4988421DD90020C9499B
S315080061008864C7484038018BC08A81420BDBC44883
S315080061102038C07A00280FD1C24948600121C048FA
S315080061202038C17208E0BE484038C18A018303E0BE
S31508006130BB484038C18A0183B9482038C07A01284B
S315080061402DD1B7482038407A012828D100230122CA
S3150800615019461846FFF7A2F900231A4619461846A3
S31508006160FFF79CF9AF4840687D210901884215D997
S315080061700020AC49486010210920C006FCF793FEB0
S3150800618080210920C006FCF78EFE0121A848FCF7ED
S315080061908AFE0021A24820384172C17210BDA0486B
S315080061A02038407A002863D110210920C006FCF760
S315080061B07AFE80210920C006FCF775FE01219C485D
S315080061C0FCF771FE00219648417200230122194608
S315080061D01846FFF763F900231A4619461846FFF7CB
S315080061E05DF990484068FF21F531884204D20421C0
S315080061F08F48FCF75AFE48E204218D48FCF753FE07
S315080062008848406889498842F5D985482038807B7E
S31508006210002817D1834840687D214901884201D268
S31508006220FDF756FE08218248FCF73DFE00217C4812
S315080062302038C17220304171817100207949086285
S3150800624008630BE040217A48FCF724FE002805D0B5
S31508006250002173484172012120384172202109200A
S31508006260C006FCF720FE7D2040016E4948600CE21E
S315080062706B48407A0300FEF7A8F806046DC8FDFCD3
S31508006280FB6C0021664841718171002065490862EE
S3150800629008630023012219461846FFF7FFF8002372
S315080062A01A4619461846FFF7F9F85D484038C18A74
S315080062B081832030C079012809D15A4800695D498F
S315080062C0884203D9002156482038C17166E75548E7
S315080062D040687D210901884223D900215048C171AF
S315080062E02038807B002802D14E49486002E0524897
S315080062F04C49486040214E48FCF7CCFD00280BD19C
S31508006300FDF7E6FD08214A48FCF7CDFD7E20FDF79E
S31508006310F5FF1E20FCF790FA04214548FCF7C3FD5B
S3150800632017E020210920C006FCF7BFFD08214048D8
S31508006330FCF7BBFD3B484068FF21F531884208D988
S315080063403748AC384089002803D104213848FCF77F
S31508006350AAFD99E133484068FF21F531884204D205
S3150800636004213348FCF7A1FD03E004213048FCF77B
S315080063709AFD2C4948687D21C900FBF7CBFA2328EA
S3150800638023D2284948687D21C900FBF7C3FA192892
S315080063901BD923484038818AFF386D3840888142A6
S315080063A007DA1F484038C18AFF386D38408881426D
S315080063B01ADB1B488079012816D100201949486044
S315080063C0C8610221164841720EE0164948687D21C7
S315080063D0C900FBF79FFA232806D300201149486015
S315080063E0C86102210E4841720E4A54325188FF3262
S315080063F06D32D08A01231A46FFF750F800231A4651
S3150800640019461846FFF74AF83EE106484068FF2154
S31508006410F531884212D204210548FCF746FD11E001
S31508006420C0030020C001002070110100B80B000055
S315080064300004004888130000C40900000421954898
S31508006440FCF731FD94484168543000897D22D2001A
S315080064505043814214D2904A54325188FF326D32E9
S31508006460D08A01231A46FFF719F800231A4602E0D4
S3150800647098E055E011E019461846FFF70FF80BE0CB
S315080064800021864801740020834948600121834819
S315080064904173032120304172F6E080482038C08AD3
S315080064A0FF217D31884204DC7C482038808A884276
S315080064B00CDD0023012219461846FEF7EFFF0023DC
S315080064C01A4619461846FEF7E9FF28E07249486851
S315080064D07D21C900FBF71EFA6F4954314989884264
S315080064E010D26D4A54329188FF326D32D08A012318
S315080064F01A46FEF7D3FF00231A4619461846FEF732
S31508006500CDFF0CE065482038818AC18300206249A6
S315080065104860002161480174042120304172B3E0CB
S315080065205E482038C08AFF217D31884204DC5B48FA
S315080065302038808A88420CDD002301221946184635
S31508006540FEF7ACFF00231A4619461846FEF7A6FFC3
S3150800655027E0514948687D21C900FBF7DBF94E4918
S315080065605431098A0F39884214D24B4A5432D18998
S31508006570FF326D32908A01230022FEF78FFF464ACA
S315080065805432D188FF326D32D08A01231A46FEF77B
S3150800659085FF06E000204049486005213F48203035
S315080065A0417271E03C484068FF21F531884204D2C7
S315080065B004213848FCF779FC0FE037484068FF218A
S315080065C0F531884209D9344840684B21C9008842C8
S315080065D003D204212F48FCF766FC2F48406830494F
S315080065E088422DD22D482038C08AFF217D31884225
S315080065F004DC2A482038808A88420CDD00230122E0
S3150800660019461846FEF74AFF00231A461946184641
S31508006610FEF744FF37E0204A5432D189FF326D3203
S31508006620908A01230022FEF739FF1B4A5432D1888B
S31508006630FF326D32D08A01231A46FEF72FFF22E079
S3150800664004211448FCF731FC134840681449C83142
S31508006650884218D300201049486000210F4820308E
S315080066604172203841720023012219461846FEF766
S3150800667015FF00231A4619461846FEF70FFF042190
S315080066800448FCF710FC00BF00BF7E20FDF736FE6D
S3150800669000BF83E500040048C0010020A0030020D5
S315080066A0A4380000C4660008C000002000010000ED
S315080066B060440008C4670008C001002040080000C4
S315080066C07044000800000000000000000000000000
S315080066D000000000000000000000000000000000AC
S315080066E0000000000000000000000000000000009C
S315080066F0000000000000010203040102030406076B
S315080067000809000000A24A0400000000000000007A
S315080067100102030406070809000000000000000043
S315080067200000000000000000040000000100000056
S31508006730000000000000000000000000000000004B
S31508006740000000000000000000000000000000003B
S31508006750000000000000000000000000000000002B
S31508006760000000000000000000000000000000001B
S3150800677000011058594C4C30313132787878787895
S31508006780787878CB7E00011058594C4C303131322C
S31508006790787878787878787804013205054C4C3022
S315080067A031310614594132303035323848343530B3
S315080067B034324178787878787D5D7E000000000074
S309080067C000000000C7
S705080018C515
